:020000040800F2
:100000008805002029020008A71500089F15000890
:10001000A315000821040008151A000800000000BC
:10002000000000000000000000000000AB15000808
:100030002504000800000000A9150008AD150008FF
:100040004D0200084D0200084D0200084D02000854
:100050004D0200084D020008290400084D02000866
:100060003D04000851040008650400084D02000822
:100070004D0200084D0200084D0200084D02000824
:100080004D0200084D0200084D0200084D02000814
:100090004D0200084D0200084D0200084D02000804
:1000A0004D0200084D0200084D0200084D020008F4
:1000B0004D0200084D0200084D0200084D020008E4
:1000C0004D0200084D0200084D0200084D020008D4
:1000D0004D020008C51900084D0200084D02000835
:1000E0004D0200084D0200084D0200084D020008B4
:1000F0004D0200084D0200084D0200084D020008A4
:100100004D0200084D0200084D0200084D02000893
:100110004D0200084D0200084D0200084D02000883
:100120004D0200084D0200084D0200084D02000873
:100130004D0200084D0200084D0200084D02000863
:100140004D0200084D0200084D0200084D02000853
:100150004D0200084D0200084D0200084D02000843
:100160004D0200084D0200084D0200084D02000833
:100170004D0200084D0200084D020008000000007A
:100180004D0200084D02000800F002F800F03CF8B3
:100190000AA090E8000C82448344AAF10107DA45E2
:1001A00001D100F031F8AFF2090EBAE80F0013F0F8
:1001B000010F18BFFB1A43F0010318474C1D000044
:1001C0006C1D0000103A24BF78C878C1FAD85207D5
:1001D00024BF30C830C144BF04680C6070470000C1
:1001E0000023002400250026103A28BF78C1FBD840
:1001F000520728BF30C148BF0B6070471FB501F0E0
:1002000071FE1FBD10B510BD00F0D7F81146FFF705
:10021000F5FF01F0B7FD00F0F5F803B4FFF7F2FFCA
:1002200003BC01F015FC00000C48016841F47001AA
:1002300001600B4880470B480047FEE7FEE7FEE7FA
:10024000FEE7FEE7FEE7FEE7FEE7FEE7FEE700006B
:1002500005480649044A064B7047000088ED00E057
:10026000B5150008890100088801002088050020D4
:1002700088010020704753EA020C00F069802DE9E4
:10028000F04B4FF00006002B1FBFB3FA83F503FAC3
:1002900005F424FA05F65E4012BF1643B2FA82F561
:1002A00002FA05F4C5F120051EBF22FA05FC44EA56
:1002B0000C04203556EA044C4FEA144418BF641C61
:1002C0004FF000084FF00009904271EB030C39D356
:1002D000002919BFB1FA81F701FA07F6B0FA80F7E1
:1002E00000FA07F6C7F120071EBF20FA07FC46EA0E
:1002F0000C062037B6FBF4FCA7EB0507103F07F010
:100300001F0BCBF120060CFA0BFB2CFA06F644BFB0
:10031000B3460026202FA4BF5E464FF0000B5BEAD9
:10032000060C08BF4FF0010B19EB0B09ABFB027C6D
:1003300048EB0608C01B06FB02CC0BFB03CC71EBA1
:100340000C01C1E70B46024641464846BDE8F08B2A
:1003500013B54FF000004FF00001AFF30080BDE88F
:100360001C4070474FF0000200B513469446964675
:10037000203922BFA0E80C50A0E80C50B1F12001B8
:10038000BFF4F7AF090728BFA0E80C5048BF0CC066
:100390005DF804EB890028BF40F8042B08BF7047C4
:1003A00048BF20F8022B11F0804F18BF00F8012B36
:1003B00070477047704770477047754600F02CF8DB
:1003C000AE4605006946534620F00700854618B042
:1003D00020B5FFF73DFFBDE820404FF000064FF08D
:1003E00000074FF000084FF0000B21F00701AC466A
:1003F000ACE8C009ACE8C009ACE8C009ACE8C00989
:100400008D46704710B50446AFF300802046BDE826
:100410001040FFF702BF000000487047280100208D
:1004200000BFFEE77047000010B5012000F0DEF8C5
:1004300001200149086010BD143C014010B50420A2
:1004400000F0D4F804200149086010BD143C0140BC
:1004500010B5082000F0CAF808200149086010BD56
:10046000143C014010B5102000F0C0F810200149E4
:10047000086010BD143C014070B50446A56D00F045
:10048000E3F9064694F83500022808D0802060651C
:1004900000BF002084F8340000BF012070BD206838
:1004A000006820F01600216808602068406920F08C
:1004B000800021684861206C08B9A06C28B12068D0
:1004C000006820F00800216808602068006820F0BB
:1004D0000100216808600FE000F0B6F9801B0528D4
:1004E0000AD92020606500BF002084F8340000BFD6
:1004F000032084F83500D1E72068006800F001008F
:100500000028E9D194F85C103F208840A86000BF23
:10051000002084F8340000BF012084F8350000205A
:10052000BCE7014691F83500022803D080204865D9
:1005300001207047052081F835000868006820F028
:1005400001000A6810600020F3E7000010B50446BF
:10055000142001F0B7FA012C32D0042C1CD0082C46
:100560000DD0102C39D110211D4800F04FF928B9B9
:1005700000BF61011B4800F051F900BF2EE00821C7
:10058000174800F043F930B900BF4FF480611548B7
:1005900000F044F900BF21E00421114800F036F9D1
:1005A00068B900BF4FF480610E4800F037F900BF12
:1005B00000BF4FF400710B4800F030F900BF0DE0B0
:1005C0000121094800F022F9012805D100BF0102EC
:1005D000044800F023F900BF00E000BF00BF10BDD9
:1005E00000100240001402400000024010B5044612
:1005F00004480068204020B1024804602046FFF70C
:10060000A5FF10BD143C0140F8B502460B4600257D
:10061000002400200021DEE0012606FA01F51E6814
:1006200006EA0504AC4275D11E7906F00306012ED8
:1006300004D01E7906F00306022E13D190684F00F5
:100640000326BE40B0434F00DE68BE40304390609A
:10065000506801268E40B0431E79C6F300168E40C6
:10066000304350601E7906F00306032E09D0D0688F
:100670004F000326BE40B0434F009E68BE4030434B
:10068000D0601E7906F00306022E13D1CF0802F1C6
:10069000200656F827004E07F70E0F26BE40B0433F
:1006A0004F07FF0E1E69BE403043CF0802F12006FF
:1006B00046F8270010684F000326BE40B0431E795D
:1006C00006F003064F00BE40304310605E6806F03F
:1006D0008056B6F1805F7DD100BF00260096404E67
:1006E000366846F480463E4F3E603E46366806F425
:1006F0008046009600BF00BF3A4E8F0856F827008C
:100700008E07370F0F26BE40B043374EB24202D19C
:10071000002624E05EE0354EB24201D101261EE003
:10072000334EB24201D1022619E0324EB24201D11B
:10073000032614E0304EB24201D104260FE02F4EC2
:10074000B24201D105260AE02D4EB24201D1062661
:1007500005E02C4EB24201D1072600E008268F07A3
:100760003F0FBE4030431F4E8F0846F82700264EED
:100770003068A0435E6806F48036B6F5803F00D14D
:100780002043214E3060361D3068A0435E6806F479
:100790000036B6F5003F00D120431B4E361D3060B9
:1007A000361D3068A0435E6806F48016B6F5801FDB
:1007B00000D12043144E08363060361D3068A04307
:1007C0005E6806F40016B6F5001F00D120430E4EF9
:1007D0000C363060491C1029FFF41EAFF8BD000034
:1007E0004438024008380140000002400004024042
:1007F00000080240000C02400010024000140240B9
:1008000000180240001C0240003C014002461369EF
:100810000B400BB1012000E00020704710B5426989
:1008200021EA020302EA010443EA0443836110BDA2
:100830000AB1816101E00B048361704701480068DF
:10084000000C7047002004E0014800687047000079
:100850001000002003480068034909780844014952
:1008600008607047100000201800002010B50A48EA
:10087000006840F40070084908600846006840F4C9
:1008800080600860032000F07FF80F2000F006F879
:1008900000F02AF8002010BD003C024070B504466C
:1008A0000E4800784FF47A71B1FBF0F00C490968FA
:1008B000B1FBF0F5284600F01DFC08B1012070BD29
:1008C000102C07D200222146501E00F01EF80548C9
:1008D000046001E00120F2E70020F0E718000020AA
:1008E0000000002014000020704701460846002840
:1008F00009DB00F01F0301229A4043099B0003F12A
:10090000E023C3F8002100BF70472DE9F05F804667
:100910000D461646002701F07FF8074639462A465D
:10092000334601F00700C0F1070ABAF1040F02D9FB
:100930004FF0040A01E0C0F1070AD14600F1040AB1
:10094000BAF1070F02D24FF0000A01E0A0F1030A4A
:10095000D4464FF0010A0AFA09FAAAF1010A0AEA92
:10096000020A0AFA0CFA4FF0010B0BFA0CFBABF17E
:10097000010B0BEA030B4AEA0B042146404601F047
:1009800053F8BDE8F09F000000BF00F00702064BDF
:1009900019684FF6FF031940044B0B4343EA022149
:1009A000014B196000BF70470CED00E00000FA0534
:1009B00070B504460D460CB9012070BD584800685A
:1009C00000F00700A84209D255490D70084600689A
:1009D00000F00700A84201D00120EEE7207800F0E7
:1009E000020002281DD1207800F00400042805D15F
:1009F0004C48006840F4E0504A490860207800F014
:100A00000800082805D14748006840F4604045497F
:100A100008604448006820F0F000A168084341499C
:100A20000860207800F00100A8B36068012807D1B1
:100A30003C4808380068C0F34040B8B90120BCE722
:100A40006068022802D06068032807D1354808385A
:100A50000068C0F3406048B90120AEE7314808386B
:100A60000068C0F3400008B90120A6E72D480068DF
:100A700020F00300616808432A490860FFF7E4FE9C
:100A8000064609E0FFF7E0FE801B41F2883188420C
:100A900002D9032091E707E02248006800F00C002B
:100AA0006168B0EB810FEDD11D48006800F00700D0
:100AB000A84209D91A490D700846006800F00700DD
:100AC000A84201D0012078E7207800F00400042833
:100AD00007D11448006820F4E050E1680843114948
:100AE0000860207800F00800082808D10D48006848
:100AF00020F46040216940EAC1000A49086000F022
:100B00003FF808490968C1F30311074A515CC8401E
:100B10000649086006480068FFF7C0FE00204CE761
:100B2000003C024008380240EE1E00080000002091
:100B300014000020014800687047000000000020F9
:100B400000B5FFF7F7FF04490968C1F38221034AA2
:100B5000515CC84000BD000008380240FE1E00087D
:100B600000B5FFF7E7FF04490968C1F34231034AC2
:100B7000515CC84000BD000008380240FE1E00085D
:100B80002DE9F047002400250026A14625480068ED
:100B900000F00C0020B1042805D008283AD105E067
:100BA000DFF8849039E0DFF8849036E01D48001FBC
:100BB000006800F03F041B48001F006800F480003C
:100BC00078B11A481749091F0968C1F38811A0FBB9
:100BD00001700146224600233846FFF74CFB0546CC
:100BE0000EE011480F49091F0968C1F38811A0FBE5
:100BF00001700146224600233846FFF73CFB0546BC
:100C00000848001F0068C0F30140401C4600B5FBC7
:100C1000F6F902E0DFF8109000BF00BF4846BDE8DB
:100C2000F0870000083802400024F40000127A0027
:100C3000F8B504460CB90120F8BD207800F0010099
:100C4000002874D0F948006800F00C0004280DD08A
:100C5000F648006800F00C00082813D1F348001F84
:100C6000006800F48000B0F5800F0BD1EF48083821
:100C70000068C0F34040002859D06068002856D171
:100C80000120D9E700BF6068B0F5803F08D1E74890
:100C90000838006840F48030E449083908601EE0F4
:100CA0006068B0F5A02F0DD1E0480838006840F426
:100CB0008020DE49083908600846006840F480302A
:100CC00008600CE0D9480838006820F48030D74923
:100CD000083908600846006820F48020086000BFDA
:100CE000606890B1FFF7B0FD054606E0FFF7ACFD88
:100CF000401B642801D903209EE7CC4808380068CF
:100D0000C0F340400028F1D011E0FFF79DFD0546FB
:100D100006E0FFF799FD401B642801D903208BE70B
:100D2000C24808380068C0F340400028F1D120785C
:100D300000F0020002285FD1BC48006800F00C00FF
:100D400058B1BA48006800F00C0008281CD1B74818
:100D5000001F006800F48000B0B9B448083800688B
:100D6000C0F3400020B1E068012801D0012063E712
:100D7000AE480838006820F0F800216940EAC10058
:100D8000AA490839086037E0E06800B30120A849A3
:100D90000860FFF759FD054606E0FFF755FD401BCB
:100DA000022801D9032047E7A04808380068C0F3AB
:100DB00040000028F1D09D480838006820F0F80075
:100DC000216940EAC10099490839086014E000200F
:100DD00097490860FFF738FD054606E0FFF734FD48
:100DE000401B022801D9032026E7904808380068F4
:100DF000C0F340000028F1D1207800F00800082856
:100E00002CD16069A8B101208A490860FFF71CFD58
:100E1000054606E0FFF718FD401B022801D9032014
:100E20000AE782486C300068C0F340000028F1D027
:100E300014E000207F490860FFF706FD054606E044
:100E4000FFF702FD401B022801D90320F4E6774892
:100E50006C300068C0F340000028F1D1207800F029
:100E60000400042870D1002770483830006800F072
:100E7000805090B900BF002000906C483830006866
:100E800040F080506949383108600846006800F039
:100E90008050009000BF00BF01276748006800F441
:100EA0008070B0B96448006840F48070624908609E
:100EB000FFF7CAFC054606E0FFF7C6FC401B022808
:100EC00001D90320B8E65C48006800F4807000286F
:100ED000F2D000BFA068012808D1544868300068EB
:100EE00040F001005149683108601DE0A068052804
:100EF0000DD14E486830006840F004004B4968311D
:100F000008600846006840F0010008600CE04748AF
:100F10006830006820F001004449683108600846E4
:100F2000006820F00400086000BFA068A8B1FFF7C7
:100F30008BFC054609E0FFF787FC401B41F2883136
:100F4000884202D9032077E626E0384868300068F6
:100F5000C0F340000028EED013E0FFF775FC054613
:100F600008E0FFF771FC401B41F28831884201D94B
:100F7000032061E62D4868300068C0F34000002877
:100F8000EFD1012F07D129483830006820F0805078
:100F900026493831086000BFA069002845D02348A1
:100FA000006800F00C0008285DD0A069022845D137
:100FB00000201F490866FFF747FC054606E0FFF7DB
:100FC00043FC401B022801D9032035E617480838A6
:100FD0000068C0F340600028F1D1D4E9070108435C
:100FE000616A40EA81110122A06AC2EB500041EA25
:100FF00000412C20005D41EA00600C49091F086097
:1010000001200B490866FFF71FFC054606E0FFF7C5
:101010001BFC401B022801D903200DE603480838B9
:101020000068C0F340600028F1D049E00838024071
:1010300000004742800E47420070004000202149D6
:101040000866FFF701FC054606E0FFF7FDFB401BC5
:10105000022801D90320EFE51B480068C0F3406077
:101060000028F2D12CE0A069012800D1E4E516485F
:10107000001D0668A069012820D006F48001E069FF
:1010800081421BD106F03F01206A814216D147F60A
:10109000C0703040616AB0EB811F0FD106F440315F
:1010A0000122A06AC2EB5000B1EB004F06D106F05E
:1010B00070612C20005DB1EB006F01D00120BBE519
:1010C0000020B9E50000474200380240042808D15A
:1010D0004FF0E021096941F004014FF0E022116175
:1010E00007E04FF0E021096921F004014FF0E02210
:1010F0001161704770B504462546681EB0F1807FC7
:1011000001D301200FE0681E4FF0E02148610F215C
:101110004FF0FF3000F088FC00204FF0E0218861A4
:1011200007200861002070BD70477047014600220B
:10113000002391F83D2091F83E3042EA03007047C9
:101140002DE9F84F0446206805682068C6682068C5
:1011500047694FF00009CA4605F00F09B9F1000FC1
:101160000AD105F0200038B106F0200020B1204659
:1011700000F05FFABDE8F88FB9F1000F72D007F008
:10118000010018B906F4907000286BD005F001003A
:1011900030B106F4807018B1206C40F0010020647A
:1011A00005F0040030B107F0010018B1206C40F0E8
:1011B0000200206405F0020030B107F0010018B110
:1011C000206C40F00400206405F0080048B106F0EF
:1011D000200010B907F0010018B1206C40F00800A1
:1011E0002064206C70B305F0200028B106F02000C8
:1011F00010B1204600F01DFA20684069C0F3801A43
:10120000206C00F0080010B9BAF1000F23D020467E
:1012100000F0E4F92068406900F04000402816D151
:101220002068406920F0400021684861A06B50B1FF
:101230005648A16B0865A06BFFF773F910B1A06B5E
:10124000016D88470CE02046FFF76FFF08E020465D
:10125000FFF76BFF04E02046FFF767FF00202064E4
:1012600088E7FFE7206B012879D105F010000028FE
:1012700075D006F01000002871D000BF002000904B
:1012800020680068009020684068009000BF00BFA0
:101290002068406900F04000402839D1A06B006808
:1012A00040681FFA80F8B8F1000F30D0A08D40459B
:1012B0002DDDA4F82E80A06BC069B0F5807F1FD013
:1012C0002068C06820F480702168C8602068406988
:1012D00020F00100216848612068406920F040004A
:1012E00021684861202084F83E00002020632068A7
:1012F000C06820F010002168C860A06BFFF7BCF840
:10130000A08DE28D801A81B22046FFF70DFF31E7F4
:10131000A08DE18D401A1FFA80F8E08DE8B1B8F198
:10132000000F1AD02068C06820F490702168C8604F
:101330002068406920F0010021684861202084F87D
:101340003E00002020632068C06820F01000216863
:10135000C86041462046FFF7E7FE0BE7FFE705F0D0
:10136000800030B106F0800018B1204600F0F9FA94
:1013700000E705F0400030B106F0400018B120460B
:1013800000F047F9F6E600BFF4E60000C9150008D2
:1013900010B504460CB9012010BDA06900B100E0F1
:1013A00000BF94F83D0028B9002084F83C00204696
:1013B00000F028F8242084F83D002068C06820F45C
:1013C00000502168C860204600F092F9206800694A
:1013D00020F49040216808612068406920F02A00CC
:1013E000216848612068C06840F400502168C860E6
:1013F00000202064202084F83D0084F83E00002076
:10140000CAE7000010B586B004462E49206888421D
:1014100055D100BF00BF002000902B48006840F06D
:101420001000294908600846006800F0100000908C
:1014300000BF00BF00BF00BF00BF002000902248D7
:101440001438006840F001001F491439086008464C
:10145000006800F00100009000BF00BF00BF00BFA7
:1014600000BF002000900846006840F001000860BE
:101470000846006800F00100009000BF00BF00BFF8
:101480004815019002200290012003900220049050
:101490000720059001A90D48FFF7B6F84FF48060CA
:1014A00001900720059001A90848FFF7ADF8252015
:1014B000FFF71BFA032211462520FFF726FA06B094
:1014C00010BD0000001001404438024000000240FE
:1014D00070B504460D46164694F83E00202816D1F5
:1014E00005B10EB9012070BD00BF94F83C00012881
:1014F00001D10220F7E7012084F83C0000BF002062
:10150000206332462946204600F008FAEBE7022025
:10151000E9E700001D4A0168914236D11C4909885B
:1015200001F4004189BB1A49098801F4804171B175
:10153000184909780A2903D00021154A118024E0AE
:101540001349098841F40041114A11801DE01149F5
:1015500009780D2906D10E49098841F480410C4AC9
:10156000118012E00B490978094A1288C2F30D0272
:10157000094B995406490988491C054A11801146AE
:101580000988C72901DD0021118070470010014042
:101590000C0000200E0000201C000020704700BF3F
:1015A000FEE700BFFEE770477047704710B5FFF7D2
:1015B00051F910BD0348006840F47000014908600B
:1015C0007047000088ED00E070B50546AC6B002068
:1015D000E085E0842046FFF7A8FD70BD0168C9687A
:1015E00021F490710268D1600168496921F001011C
:1015F00002685161016B012905D10168C96821F0B8
:1016000010010268D160202180F83E1000210163A2
:10161000704710B504462068C06820F0400021687B
:10162000C860202084F83D002046FFF7B7FF002067
:1016300010BD70B5044694F83E00222856D1A0682B
:10164000B0F5805F0CD1206950B90025A66A2068EA
:101650004068C0F308003080A06A801CA06215E0DA
:10166000A56A0026A068B0F5805F03D0A06828B9FD
:10167000206918B920684068287004E02068406834
:1016800000F07F002870A06A401CA062E08D401E20
:1016900080B2E08540BB2068C06820F0200021684F
:1016A000C8602068C06820F480702168C860206825
:1016B000406920F0010021684861202084F83E0044
:1016C000206B01280AD12068C06820F01000216832
:1016D000C860A18D2046FFF727FD02E02046FFF7F6
:1016E00019FF0020206370BD0020FCE70220FAE70C
:1016F0002DE9F84F04462068006920F44050E16865
:101700000843216808612169A068084361690843AA
:10171000E169084300902068C06849F20C61884381
:10172000009908432168C8602068406920F440702F
:10173000A16908432168486176492068884203D03E
:1017400075492068884203D1FFF70AFA814602E012
:10175000FFF7F6F98146E069B0F5004F6CD1022041
:101760006168A0FB015003461920A9FB00700146E7
:101770002A463846FEF77FFD6421B0FBF1F04FEAC0
:10178000001A02206168A0FB01510B461920A9FB39
:1017900000712A463846FEF76EFD834602206168D6
:1017A000A0FB015003461920A9FB00712A463846C8
:1017B000FEF761FD6421B0FBF1F000EBC00101EB2D
:1017C0000010ABEB8000322101EBC0006421B0FBC4
:1017D000F1F000F0F8000AEB400A02206168A0FB7B
:1017E000015003461920A9FB007001462A463846DD
:1017F000FEF741FD834602206168A0FB01500346CD
:101800001920A9FB00712A463846FEF734FD6421F1
:10181000B0FBF1F000EBC00101EB0010ABEB80007E
:10182000322101EBC0006421B0FBF1F000F00700B1
:101830005044216888606AE004206168A0FB015080
:1018400003461920A9FB007001462A463846FEF7D8
:1018500012FD824604206168A0FB01500346192056
:10186000A9FB007001462A463846FEF704FD6421B4
:10187000B0FBF1F000EBC00101EB0010AAEB80001F
:10188000322101EB00106421B0FBF1F000F0F00A0E
:1018900004206168A0FB017003461920A9FB0051D8
:1018A0003A462846FEF7E7FC6421B0FBF1F00AEB6C
:1018B000001A04206168A0FB01510B461920A9FB06
:1018C00000712A463846FEF7D6FC8346042061683C
:1018D000A0FB015003461920A9FB007001462A46CF
:1018E0003846FEF7C8FC6421B0FBF1F000EBC00104
:1018F00001EB0010ABEB8000322101EB0010642102
:10190000B0FBF1F000F00F00504421688860BDE8A2
:10191000F88F0000001001400014014010B503468C
:1019200099629A85DA8500201864222083F83E00A7
:1019300000BF002083F83C0000BF1868C06840F476
:1019400080701C68E0601868406940F001001C6805
:1019500060611868C06840F020001C68E0600020EA
:1019600010BD014691F83D00212828D18868B0F5C6
:10197000805F0BD1086948B90A6A1088C0F3080073
:101980000B685860086A801C086205E00B6A581CE6
:10199000086218780B685860C88C401E80B2C884F2
:1019A00058B90868C06820F080000B68D8600868E3
:1019B000C06840F040000B68D860002070470220EB
:1019C000FCE7000070B500240F4D1048FFF7B8FB8E
:1019D00000BF03E0641CAC4200D904E00B48FFF7F1
:1019E000A5FB2028F6D100BF002403E0641CAC4214
:1019F00000D906E0012206490448FFF769FD0028E6
:101A0000F4D100BF70BD0000FFFF0100E400002022
:101A10000E00002000BFFEE702480068C0F302206D
:101A2000704700000CED00E010B5002804DB0A0749
:101A3000130E054A135406E00A07140E034A00F079
:101A40000F031B1FD45410BD00E400E018ED00E0AC
:101A500000BF704700B587B000BF00BF00200190F5
:101A60001148006840F020000F49086008460068EF
:101A700000F02000019000BF00BF00BF8815029059
:101A80000120039004900220059002A90748FEF768
:101A9000BBFD00BF00224FF480710448FEF7C8FE72
:101AA00000BF07B000BD0000303802400014024003
:101AB00010B504460420FFF709FB0148046010BD7F
:101AC0000400002070B504464FF4077094FBF0F555
:101AD00094FBF0F100FB114603E0074800F00EF81C
:101AE0006D1E002DF9D12EB14FF47A7106FB01F075
:101AF00000F004F870BD0000603D080070B50346BA
:101B000000224FF0E02675690D4E366803FB06F49F
:101B10004FF0E026B16910E04FF0E026B06988424E
:101B20000BD0884202D20E1A324402E02E1A0E4422
:101B300032440146A24200D300E0EDE700BF70BD91
:101B40000400002000B585B000F052F8102000908D
:101B5000234801900120029069462248FEF754FD77
:101B6000082000901E4801900120029069461D48FF
:101B7000FEF74AFD042000901948019001200290D0
:101B800069461848FEF740FD012000901648019074
:101B90000220029069461548FEF736FD0222002118
:101BA0000A20FEF7B2FE0A20FEF79FFE0222012164
:101BB0000920FEF7AAFE0920FEF797FE0222114631
:101BC0000820FEF7A2FE0820FEF78FFE0222032166
:101BD0000620FEF79AFE0620FEF787FE05B000BD40
:101BE000000021100010024000001110000002400F
:101BF00000B587B000BF00BF0020019038480068E2
:101C000040F01000364908600846006800F01000F7
:101C1000019000BF00BF00BF00BF00BF00200190C7
:101C20000846006840F0100008600846006800F0B0
:101C30001000019000BF00BF00BF00BF00BF002028
:101C400001900846006840F01000086008460068EF
:101C500000F01000019000BF00BF00BF00BF00BF38
:101C6000002001900846006840F001000860084626
:101C7000006800F00100019000BF00BF00BF10200D
:101C8000029000200390012004900220059002A9F8
:101C90001448FEF7B9FC08200290002003900120B0
:101CA00004900220059002A90E48FEF7ADFC042026
:101CB000029000200390012004900220059002A9C8
:101CC0000848FEF7A1FC01200290002003900220AA
:101CD0000490059002A90448FEF796FC07B000BDE9
:101CE00030380240001002400000024000B587B0CA
:101CF00000BF00BF002001902048006840F0200095
:101D00001E4908600846006800F02000019000BFEE
:101D100000BF00BF00BF00BF002001900846006860
:101D200040F0200008600846006800F020000190A4
:101D300000BF00BF00BF481502900120039004902F
:101D40000220059002A90E48FEF75EFC4FF4806069
:101D5000029002A90A48FEF757FC00BF0122510277
:101D60000748FEF765FD00BF00BF0122910204484D
:101D7000FEF75EFD00BF07B000BD00003038024036
:101D800000140240FEF772FD0723022208214FF4DF
:101D9000A87000F01DF8A820FFF78AFE4FF4E1308C
:101DA00000F084F8FFF7A2FFFFF754FEFFF7CAFE2A
:101DB00000BF00224FF400710448FEF739FD00BF58
:101DC00003E04FF47A70FFF77DFEFAE7001402405B
:101DD0002DE9F04192B080460C4615461E4600277C
:101DE000302106A8FEF7BEFA142101A8FEF7BAFAC0
:101DF00000BF002000902A48006840F08050284929
:101E000008600846006800F08050009000BF00BFE6
:101E100000BF002000902348006840F48040214922
:101E200008600846006800F48040009000BF00BFD2
:101E3000012006900004079002200C9041050D91AE
:101E4000CDF83C800E941095119606A8FEF7F0FE92
:101E500007461FB1012012B0BDE8F0810F200190AC
:101E600002200290002003904FF4A05004904FF401
:101E700080500590052101A8FEF79AFD07460FB195
:101E80000120E8E7FEF7DAFC41F20101884205D1C2
:101E90000548006840F48070034908600020DAE7D4
:101EA0004038024000700040003C024010B504463B
:101EB00009480A4908600846446000218160C16001
:101EC000016181610C214161FFF762FA012204493D
:101ED0000248FFF7FDFA10BD00100140E4000020A9
:101EE0000E0000204FF04070E1EE100A7047000035
:101EF00000000000000001020304060708090000BA
:101F00000000010203040000281F00080000002058
:101F10001C000000C4010008441F00081C00002031
:101F20006C050000E00100080024F400000000003F
:101F30000000000000000000000000001000000091
:041F4000010000009C
:040000050800018965
:00000001FF
